:1000000023C23DC23CC23BC23AC239C238C237C227
:1000100036C230C334C233C232C231C230C22FC240
:100020002EC22DC22CC2464D00D0E0E4E8EE205294
:100030004441353830376D002020C0EBFCF4E0201F
:10004000D0E0E4E8EE20002020D0E0E4E8EE20CC90
:10005000E8F0202020002020C1E5EBEEF0F3F1F1E4
:10006000EAEEE52000C4F3F8E5E2EDEEE520F0E08D
:10007000E4E8EE002020D0E0E4E8EE20C1E820DD56
:10008000E920002020D0E0E4E8F3F120464D2020D4
:1000900020002020202020526F6B73202020202061
:1000A000002020D0E0E4E8EE20CECDD220202000B9
:1000B000202020CFE8EBEEF220464D20202000202B
:1000C0002020554E49535441522020202000D0F387
:1000D000F1F1EAEEE520F0E0E4E8EE200020CDEEDC
:1000E000E2EEE520F0E0E4E8EE20200020CCE5EBB5
:1000F000EEE4E8E820E2E5EAE02000202020DEEC63
:10010000EEF020464D202020200020D0E0E4E8EE54
:1001100020CCE8EDF1EA2020002020202020202023
:100120002020202020202000000000000000005F90
:1001300000000007000700147F147F14242A7F2A80
:10014000124C2C10686436495522500005030000FB
:10015000001C2241000041221C0014083E08140823
:10016000083E080800005030001010101010006009
:1001700060000020100804023E5149453E00427FC5
:10018000400042615149462141454B311814127FCC
:100190001027454545393C4A494930017109050355
:1001A0003649494936064949291E003636000000BD
:1001B000563600000814224100141414141400418F
:1001C0002214080201510906324979413E7E11117B
:1001D000117E7F494949363E414141227F414122BA
:1001E0001C7F494949417F090909013E4149497A32
:1001F0007F0808087F00417F41002040413F017F88
:10020000081422417F404040407F020C027F7F045F
:1002100008107F3E4141413E7F090909063E415198
:10022000215E7F09192946464949493101017F016B
:10023000013F4040403F1F2040201F3F4038403F8B
:1002400063140814630708700807615149454300A7
:100250007F41410002040810200041417F00040258
:100260000102044040404040000102040020545478
:1002700054787F48444438384444442038444448FF
:100280007F3854545418087E0901020C5252523ED1
:100290007F0804047800447D40002040443D007FF6
:1002A0001028440000417F40007C041804787C083A
:1002B00004047838444444387C1414140808141492
:1002C000187C7C080404084854545420043F4440DB
:1002D000203C4040207C1C2040201C3C4030403CC6
:1002E00044281028440C5050503C4464544C440062
:1002F0000836410000007F00000041360800080475
:10030000081008FFFFFFFFFF7C1211127C7F494994
:1003100049317F494949367F01010101603F213F51
:10032000607F4949494177087F087722414949362A
:100330007F1008047F7E1009047E7F08142241404C
:100340003E01017F7F020C027F7F0808087F3E414B
:1003500041413E7F0101017F7F090909063E41417C
:10036000412201017F0101074848483F0E117F11DA
:100370000E63140814633F20203F60070808087FBD
:100380007F407E407F3F203F207F017F4848307F75
:100390004830007F007F484830224149493E7F086D
:1003A0003E413E462919097F20545454783C4A4A1C
:1003B0004A317C545428007C04040C00603C243CEA
:1003C0006038545454186C107C106C0044545428F9
:1003D0007C2010087C7C2112097C7C102844004081
:1003E0003804047C7C0810087C7C1010107C384495
:1003F0004444387C0404047C7C14141408384444B9
:10040000440004047C04040C5050503C08147C1438
:100410000844281028443C20203C600C1010107C1C
:100420007C407C407C3C203C207C047C5050207CE8
:100430005020007C007C50502028445454387C10BC
:10044000384438485434147C11241FBECFE5D4E01E
:10045000DEBFCDBF11E0A0E6B0E0E2E4FCE102C007
:1004600005900D92AC36B107D9F713E0ACE6B1E0D8
:1004700001C01D92AC38B107E1F727D2E0CBC0CD67
:10048000A59A8AE0982F9A95F1F7A49A982F9A95B1
:10049000F1F7A598982F9A95F1F7A4988A95F1F716
:1004A00010926C019C9905C080916C018F5F8093C4
:1004B0006C019D9905C080916C018F5F80936C01E8
:1004C0008AE0982F9A95F1F7982F9A95F1F7982F3F
:1004D0009A95F1F78A95F1F70895A498A598AC98A4
:1004E000AD98CEDFCDDF0895A49A8AE0982F9A9533
:1004F000F1F7A59A8A95F1F70895A4988AE0982FC4
:100500009A95F1F7A598982F9A95F1F7A49A982FB4
:100510009A95F1F7A59A8A95F1F7089520E04AE0B7
:1005200087FD02C0A49A01C0A4983AE0942F9A953E
:10053000F1F7A598942F9A95F1F7A59A2F5F283097
:1005400011F0880FEDCFA498832F8A95F1F7A59825
:10055000832F8A95F1F783B3A59A90E024E09695CE
:1005600087952A95E1F781700895A49820E030E0FE
:100570004AE0330FA598942F9A95F1F79C99316032
:10058000A59A942F9A95F1F72F5F283091F7882339
:1005900011F4A49A01C0A4988AE0982F9A95F1F7D3
:1005A000A598982F9A95F1F7A59A8A95F1F7A498AE
:1005B000832F089599DF80E2B1DF80916E01AEDF75
:1005C00080916F01ABDF80917001A8DF8091710194
:1005D000A5DF80917201A2DF809173019FDF80917E
:1005E00074019CDF8091750199DF8091760196DF1F
:1005F00047DF089582ED80936E018DE880936F014F
:10060000109270011092710182E080937201109239
:10061000730188E0809374018FE880937501CADFCD
:10062000089590917501982B90937501C3DF0895FB
:1006300090916E019160880F982B90936E01BADFB4
:1006400008950895865693409C01369527953695D2
:100650002795209370018295880F880F807C806198
:1006600080937101A7DF80E065E041E029E131E09E
:10067000DCD408951F920F920FB60F9211242F937E
:100680003F934F935F936F937F938F939F93AF931A
:10069000BF93EF93FF936AD220D3FF91EF91BF9165
:1006A000AF919F918F917F916F915F914F913F910A
:1006B0002F910F900FBE0F901F9018951F93182F1A
:1006C000813079F48CE993E0BDDF8CE993E090937D
:1006D00061008093600080E065E041E02AE031E065
:1006E000EDC0823079F489EA93E0ACDF89EA93E0E7
:1006F000909361008093600080E065E041E02BEF23
:1007000030E0DCC0833079F482EC93E09BDF82EC54
:1007100093E0909361008093600080E065E041E0A9
:100720002CEE30E0CBC0843079F488ED93E08ADFA2
:1007300088ED93E0909361008093600080E065E035
:1007400041E02DED30E0BAC0853079F48DED93E0D5
:1007500079DF8DED93E0909361008093600080E0FD
:1007600065E041E02EEC30E0A9C0863079F483EEFC
:1007700093E068DF83EE93E09093610080936000E4
:1007800080E065E041E02FEB30E098C0873079F4FD
:1007900084EF93E057DF84EF93E0909361008093C0
:1007A000600080E065E041E020EB30E087C0883009
:1007B00079F489EF93E046DF89EF93E0909361004D
:1007C0008093600080E065E041E021EA30E076C09F
:1007D000893079F48DEF93E035DF8DEF93E09093DE
:1007E00061008093600080E065E041E022E930E054
:1007F00065C08A3079F48DE094E024DF8DE094E0E8
:10080000909361008093600080E065E041E023E820
:1008100030E054C08B3079F486E194E013DF86E158
:1008200094E0909361008093600080E065E041E097
:1008300024E730E043C08C3079F481E294E002DFB9
:1008400081E294E0909361008093600080E065E035
:1008500041E025E630E032C08D3079F486E294E064
:10086000F1DE86E294E0909361008093600080E086
:1008700065E041E026E530E021C08E3079F48FE27A
:1008800094E0E0DE8FE294E090936100809360005A
:1008900080E065E041E027E430E010C08F3079F47B
:1008A00087E394E0CFDE87E394E090936100809348
:1008B000600080E065E041E028E330E0B6D380E00E
:1008C00090E0612F9FD91F9108952F923F924F92F0
:1008D0005F926F927F928F929F92AF92BF92CF92D0
:1008E000DF92EF92FF920F931F93DF93CF93CDB7D9
:1008F000DEB764970FB6F894DEBF0FBECDBFAED59E
:10090000ECDD2DD177DE83B7856083BF89B7816049
:1009100089BF12BE80E090E06DD980936200CEDE88
:1009200085D57894F8E32F2EF4E03F2EE6EFAE2E37
:10093000EFEFBE2E7CE9872E7FEF972E68E1462EE3
:100940006CEF562E6E010894C11CD11C58EC652E1C
:10095000712C80E060E041E029E230E066D328D1EC
:1009600080936D018130B9F48091600090916100B5
:10097000019690936100809360008953944030F019
:1009800086E693E090936100809360008091600020
:100990009091610057DE80916D018230A9F48091C1
:1009A00060009091610001979093610080936000D6
:1009B0008656934020F4309261002092600080912E
:1009C0006000909161003EDE80916D01833069F49A
:1009D000809162008F5F80936200803118F081E027
:1009E000809362008091620069DE80916D018430A5
:1009F00069F480916200815080936200882319F429
:100A00008FE0809362008091620058DE4091600028
:100A1000F0906100842F9F2D68EE73E079D8E62E68
:100A200060938B03E62FF0E0EA9D8001EB9D100DB3
:100A3000FA9D100D1124842F9F2D64E670E068D874
:100A4000262F200F2093890330E0E89D8001E99D47
:100A5000100DF89D100D1124842F9F2D6AE070E079
:100A600057D8600F2A9DC0012B9D900D3A9D900D87
:100A70001124680F60938803E49DC001E59D900DEB
:100A8000F49D900D1124480F289DC001299D900DC3
:100A9000389D900D1124480F6A9D602D1124640F1C
:100AA00060938A038E2D90E0B6014AE050E08ED824
:100AB00081E063E042E096019ED28091890390E05C
:100AC000B6014AE050E082D883E063E042E096015C
:100AD00092D28091880390E0B6014AE050E076D847
:100AE00085E063E042E0960186D28BE260E241E07D
:100AF000CED28BE26FE141E0CAD28BE26EE141E0FF
:100B0000C6D28AE26FE141E0C2D28CE26EE141E0FE
:100B1000BED28CE26FE141E0BAD28CE260E241E009
:100B2000B6D28DE26FE141E0B2D280918A0390E0CB
:100B3000B6014AE050E04AD888E063E042E096011E
:100B40005AD28BE063E041E026E230E06ED280E9E9
:100B500091E0F3013197F1F70197D9F7FACE84B319
:100B6000807F84BB85B38F6085BB0895989902C050
:100B700091E00BC09A9902C093E007C0999902C016
:100B800092E003C09B9911C094E0809178018D3070
:100B900020F084E08093780105C08F5F8093780116
:100BA000833029F490937701089510927801089585
:100BB00080917701109277010895809377010895CD
:100BC00021E030E008C0A901489F9001499F300D05
:100BD000589F300D1124615070405FEF6F3F7507D3
:100BE00091F7C9010895EF92FF920F931F93CF934E
:100BF000DF937B018C01EA0121E030E00AC0C901EA
:100C0000880F991F63E0220F331F6A95E1F7280FC1
:100C1000391F415050408FEF4F3F580781F7B901BE
:100C2000882777FD8095982F2CD59B01AC01C801B2
:100C3000B70132D480D5CB0177FD03C001E010E0CD
:100C400002C00FEF1FEF089F9001099F300D189F02
:100C5000300D1124E8E8F1E04EE2C9016AE070E0ED
:100C60006BD7805D8293C9016AE070E065D7CB01E4
:100C70009B01219709F44293892B79F71C161D06D5
:100C80007CF4AE0120E304C0FC01208341505040BD
:100C9000CF01019714161506BCF3FC018EE2808388
:100CA00080818E3211F480E382930F5F1F4F11F425
:100CB0008DE28293CF01DF91CF911F910F91FF9031
:100CC000EF900895C298613011F4C19A01C0C198A3
:100CD0008FB9779BFECFC29A0895EF92FF920F9340
:100CE0001F93CF93DF93809181039091820397FFAD
:100CF00005C0109282031092810309C0885F914061
:100D000034F087EF91E09093820380938103809188
:100D100083039091840397FF05C01092840310927F
:100D2000830309C0885F914034F087EF91E090938E
:100D3000840380938303C0918103D0918203CE0109
:100D400064E570E0F9D6806860E0BCDFCE0164E560
:100D500070E0F2D6862F806460E0B4DFE090830319
:100D6000F09084038E0107571E4F06C0F801819151
:100D70008F0161E0A7DF2196EC16FD06BCF787EF37
:100D800091E09093820380938103109284031092E8
:100D9000830310928703DF91CF911F910F91FF90F2
:100DA000EF9008951F93182F81E260E08BDF812F71
:100DB000806860E087DF80E260E084DF1F91089553
:100DC000982F8E3090F4663080F424E5629F900175
:100DD000112486E0989FC0011124280F391F3093F9
:100DE00086032093850380E0089581E00895CF92E3
:100DF000DF92EF92FF920F931F93CF93DF93282FF1
:100E0000A0918503B0918603809181039091820324
:100E1000A817B90724F4B0938203A0938103462F47
:100E20004052403630F0603C10F44FE502C0462F8F
:100E300040562130B9F485E0489FF0011124E85D67
:100E4000FE4FED01C757DE4F90E08491880F8993E4
:100E50009F5F31969530C9F71596B0938603A0939E
:100E600085039CC0223009F099C09D012455304073
:100E700080918103909182032817390724F43093DD
:100E800082032093810337FF02C081E0ABC085E07D
:100E9000489F80011124085D1E4FE901C757DE4FAE
:100EA00049E8E42E41E0F42EEA0EFB1E3FE3C32E98
:100EB00031E0D32ECA0EDB1EF8016491660F462F77
:100EC00050E0CA0184709070FC01EE0FFF1FE80F24
:100ED000F91FEE0FFF1FEE0FFF1F9A0122703070F7
:100EE000C901880F991F820F931F880F991FE82B44
:100EF00048705070CA01880F991F840F951F53E0E6
:100F0000880F991F5A95E1F7E82B62956F7070E092
:100F1000CB01847090709C01220F331F280F391F62
:100F2000220F331F220F331FAB0142705070CA01D2
:100F3000880F991F840F951F880F991F282BAB01CD
:100F400048705070CA01880F991F840F951F33E0B5
:100F5000880F991F3A95E1F7282B61707070CB01CB
:100F6000880F991F860F971F282BE883E983F701C5
:100F7000208321830F5F1F4F229682E090E0E80ECE
:100F8000F91ECC15DD0509F097CFCD010B9668EF62
:100F900071E0D2D5909386038093850320918503D9
:100FA0003091860380918303909184038217930785
:100FB00024F43093840320938303F901E757FE4F11
:100FC000108291E0273F390731F410928603109286
:100FD000850382E007C02F5F3F4F30938603209345
:100FE000850380E0DF91CF911F910F91FF90EF90EB
:100FF000DF90CF9008950F931F93CF93DF93042F2B
:10100000E901DEDE10E005C0802FF1DE813041F025
:101010001F5FFE01E10FF11D60816623A9F780E0EB
:10102000DF91CF911F910F9108951F93CF93DF937D
:10103000142FE901C5DEFE01649107C0812FD7DEC0
:10104000813031F02196FE0164916623B9F780E08A
:10105000DF91CF911F910895BF92CF92DF92EF92CF
:10106000FF920F931F93D82EC62EB42EC901B8013C
:10107000A701B9DD9C018D2D6C2D4B2DBCDF1F917F
:101080000F91FF90EF90DF90CF90BF900895582F71
:10109000843508F05AC0603308F057C0862F869513
:1010A0008695869590E024E530E0829FD001839F6D
:1010B000B00D929FB00D1124A50FB11D53E0880F04
:1010C000991F5A95E1F7681BFD01E757FE4F2081F4
:1010D000442351F481E090E002C0880F991F6A9583
:1010E000E2F78095282315C0413049F481E090E073
:1010F00002C0880F991F6A95E2F7282B0AC0423078
:1011000041F481E090E002C0880F991F6A95E2F7F0
:101110002827FD01E757FE4F20838091810390919E
:101120008203A817B90724F4B0938203A093810324
:1011300080918303909184038A179B0724F4B093D2
:101140008403A093830380E0089581E008955F9273
:101150006F927F928F929F92AF92BF92CF92DF92C7
:10116000EF92FF920F931F93CF93DF93C82ED62E4B
:10117000542E622E702E022F10E0061B1109C42F70
:10118000D0E0C81BD10917FD04C0B1E08B2E912C13
:1011900006C0109501951F4F88248A94982CD7FD7E
:1011A00004C0A1E0AA2EB12C06C0D095C195DF4F96
:1011B000AA24AA94BA2C8C2D6D2D472D68DF882384
:1011C000D9F57E01EE0CFF1C000F111F0E151F0537
:1011D000C4F4C70195958795E801C81BD90B0EC0CB
:1011E000D7FD03C0D80CCE19DF09CA0C8C2D6D2D8C
:1011F000472D4DDF882301F5C00FD11FC51481F79E
:1012000017C0C80195958795E701C81BD90B0EC07B
:10121000D7FD03C0CA0CC01BD10BD80C8C2D6D2D73
:10122000472D35DF882341F4CE0DDF1DD61481F71D
:1012300081E08093870380E0DF91CF911F910F9130
:10124000FF90EF90DF90CF90BF90AF909F908F90E6
:101250007F906F905F9008959F92AF92BF92CF92D0
:10126000DF92EF92FF920F931F93982EA62EC22E1D
:1012700083E5891508F453C08FE2861708F44FC040
:10128000D42E842F880F03E0081BEE2440C01E2DAF
:10129000190DFD2CFA0C812F6F2D4C2DF8DEBA2C78
:1012A000BD18812F6B2D4C2DF2DE192D1E19812FAB
:1012B0006F2D4C2DECDE812F6B2D4C2DE8DE1D2D7E
:1012C000190DFE2CFA0C812F6F2D4C2DE0DEBA2C5F
:1012D000BE18812F6B2D4C2DDADE192D1D19812F93
:1012E0006F2D4C2DD4DE812F6B2D4C2DD0DE07FFC2
:1012F00006C00A5F8E2D880F880F080F07C0065F93
:101300008E2D8D19880F880F080FDA94E394DE1460
:101310000CF0BDCF81E08093870380E001C081E0C5
:101320001F910F91FF90EF90DF90CF90BF90AF9003
:101330009F900895DF92EF92FF920F931F93CF93A8
:10134000DF93E82E162FD02E83E58E1530F1603313
:1013500020F5641710F4FF2413C01F5FF12EF41A58
:1013600011500EC0802F6F2D4D2D91DE8823B1F4CA
:101370000F5F802F90E08C179D07A4F3F39404C0B7
:10138000CE2DD0E0C20FD11D1F1510F00E2DF1CFC4
:1013900081E08093870380E001C081E0DF91CF91FD
:1013A0001F910F91FF90EF90DF900895CF92DF9201
:1013B000EF92FF920F931F93C82EF62ED42EE22E9B
:1013C00083E58C1548F1841738F18FE2861720F1F8
:1013D000821710F1C41610F5621700F51C2D09C014
:1013E000812F6F2D402F53DE812F6E2D402F4FDE2A
:1013F0001F5FD116A8F71F2D09C08C2D612F402F1C
:1014000046DE8D2D612F402F42DE1F5FE116A8F7CB
:1014100081E08093870302C081E001C080E01F91DA
:101420000F91FF90EF90DF90CF90089588EF91E0BB
:10143000E9E8F1E0DF019C011D9221503040E1F725
:10144000109282031092810387EF91E090938403BE
:101450008093830381E0809387030895C49A87B3C0
:101460008E6387BBC498C49A80E58DB9C29A81E225
:1014700060E028DC88EC60E025DC86E060E022DCCF
:1014800083E160E01FDC80E260E01CDC8CE060E077
:1014900019DCCCDF22DC0895A0E2B0E0E1E5FAE05F
:1014A0005EC369837A838B839C832D833E834F83C2
:1014B0005887CE010196BE01675F7F4FB1D2CE0142
:1014C0000596BE016F5E7F4FABD29985923088F052
:1014D00089898230C8F0943019F4823051F404C004
:1014E000843029F4923081F483E690E0C6C09230D3
:1014F00049F420E09A858A89981321E02A87CE0151
:101500000996BBC0823049F420E09A858A899813F5
:1015100021E02A8BCE014196B0C02D843E844F84B9
:1015200058886D887E888F88988CEE24FF248701E8
:10153000AA24BB24650140E050E060E070E0E0E0F8
:10154000F0E0C10181709070892BE9F0E60CF71C86
:10155000081D191D9A01AB012A0D3B1D4C1D5D1D77
:1015600080E090E0A0E0B0E0E614F704080519057B
:1015700020F481E090E0A0E0B0E0BA01A901480FBA
:10158000591F6A1F7B1FAA0CBB1CCC1CDD1C97FEBD
:1015900008C081E090E0A0E0B0E0A82AB92ACA2AF9
:1015A000DB2A3196E032F10549F0660C771C881C85
:1015B000991C5694479437942794C3CFFA85EA89A7
:1015C0002B893C898B859C85280F391F2E5F3F4FC7
:1015D00017C0CA0181709070892B61F0169507952C
:1015E000F794E79480E090E0A0E0B0E8E82AF92AD8
:1015F0000A2B1B2B76956795579547952F5F3F4F85
:1016000077FDE7CF0CC0440F551F661F771F17FDEE
:101610004160EE0CFF1C001F111F21503040403074
:1016200090E0590790E0690790E4790760F32B8F09
:101630003C8FDB01CA018F779070A070B07080344E
:101640009105A105B10561F447FD0AC0E114F1045B
:101650000105110529F0405C5F4F6F4F7F4F4078C7
:101660001A8EFE1711F081E08A8F4D8F5E8F6F8F7B
:1016700078A383E0898FCE014996FDD0A096E2E160
:101680008AC2A8E0B0E0E6E4FBE072C29B01AC01D4
:1016900083E08983DA01C9018827B7FD83959927FB
:1016A000AA27BB27B82E211531054105510519F48C
:1016B00082E0898339C08823A9F0203080E0380790
:1016C00080E0480780E8580729F460E070E080E097
:1016D0009FEC2EC0EE24FF248701E21AF30A040BCC
:1016E000150B02C079018A018EE1C82ED12CDC8253
:1016F000CB82ED82FE820F831887C801B7016CD0C0
:1017000001971816190684F4082E04C0EE0CFF1C6D
:10171000001F111F0A94D2F7ED82FE820F831887F3
:10172000C81AD90ADC82CB82BA82CE010196A3D034
:101730002896E9E039C2ACE0B0E0E0EAFBE01FC285
:1017400069837A838B839C83CE010196BE016B5F94
:101750007F4F66D18D81823061F1823050F18430CB
:1017600021F48E81882351F12EC02F81388537FDD9
:1017700020C06E812F3131051CF06623F9F023C0A3
:101780008EE190E0821B930B29853A854B855C8521
:1017900004C056954795379527958A95D2F76623C5
:1017A000B1F050954095309521953F4F4F4F5F4F89
:1017B0000EC020E030E040E050E009C02FEF3FEFE6
:1017C0004FEF5FE704C020E030E040E050E8B901AF
:1017D000CA012C96E2E0EFC1EF92FF920F931F93A4
:1017E0007B018C0180E0E81680E0F80681E00807C4
:1017F00080E0180788F48FEFE816F1040105110561
:1018000031F028F088E090E0A0E0B0E017C080E080
:1018100090E0A0E0B0E012C080E0E81680E0F806BA
:1018200080E0080781E0180728F088E190E0A0E058
:10183000B0E004C080E190E0A0E0B0E020E230E061
:1018400040E050E0281B390B4A0B5B0B04C0169597
:101850000795F794E7948A95D2F7F701E559FF4F7A
:101860008081281B310941095109C9011F910F913C
:10187000FF90EF900895DF92EF92FF920F931F93E6
:10188000FC01E480F58006811781D180808182305F
:1018900048F480E090E0A0E1B0E0E82AF92A0A2BC1
:1018A0001B2BA5C0843009F49FC0823021F4EE24A4
:1018B000FF24870105C0E114F1040105110519F4A5
:1018C000E0E0F0E096C0628173819FEF62387907B3
:1018D0000CF05BC022E83FEF261B370B2A313105A5
:1018E0002CF020E030E040E050E02AC0B801A70131
:1018F000022E04C076956795579547950A94D2F7BE
:1019000081E090E0A0E0B0E004C0880F991FAA1F1A
:10191000BB1F2A95D2F70197A109B1098E219F21FA
:10192000A023B1230097A105B10521F081E090E04B
:10193000A0E0B0E09A01AB01282B392B4A2B5B2B9E
:10194000DA01C9018F779070A070B0708034910572
:10195000A105B10539F427FF09C0205C3F4F4F4F67
:101960005F4F04C0215C3F4F4F4F5F4FE0E0F0E01E
:101970002030A0E03A07A0E04A07A0E45A0710F0A0
:10198000E1E0F0E079018A0127C06038710564F573
:10199000FB01E158FF4FD801C7018F779070A0700D
:1019A000B07080349105A105B10539F4E7FE0DC092
:1019B00080E490E0A0E0B0E004C08FE390E0A0E01D
:1019C000B0E0E80EF91E0A1F1B1F17FF05C0169591
:1019D0000795F794E794319687E016950795F79465
:1019E000E7948A95D1F705C0EE24FF248701EFEF35
:1019F000F0E06E2F679566276795902F9F77D794B5
:101A0000DD24D7948E2F8695492F462B582F5D299C
:101A1000B701CA011F910F91FF90EF90DF900895D9
:101A2000FC01DB01408151812281622F6F7770E0E0
:101A3000221F2227221F9381892F880F822B282F74
:101A400030E0991F9927991F11969C9311972115A2
:101A50003105A9F5411551056105710511F482E0C3
:101A600037C082E89FEF13969C938E9312979A014A
:101A7000AB0167E0220F331F441F551F6A95D1F752
:101A800083E08C930DC0220F331F441F551F129605
:101A90008D919C911397019713969C938E93129717
:101AA000203080E0380780E0480780E4580758F38A
:101AB00014962D933D934D935C93179708952F3F64
:101AC000310579F4411551056105710519F484E07A
:101AD0008C93089564FF03C081E08C9312C01C9224
:101AE00010C02F57304013963C932E93129783E0EB
:101AF0008C9387E0440F551F661F771F8A95D1F797
:101B0000706414964D935D936D937C93179708952D
:101B1000AA1BBB1B51E107C0AA1FBB1FA617B70713
:101B200010F0A61BB70B881F991F5A95A9F780952F
:101B30009095BC01CD01089597FB092E07260AD088
:101B400077FD04D0E5DF06D000201AF4709561958A
:101B50007F4F0895F6F7909581959F4F08952F92A6
:101B60003F924F925F926F927F928F929F92AF922D
:101B7000BF92CF92DF92EF92FF920F931F93CF937A
:101B8000DF93CDB7DEB7CA1BDB0B0FB6F894DEBF11
:101B90000FBECDBF09942A88398848885F846E8437
:101BA0007D848C849B84AA84B984C884DF80EE8081
:101BB000FD800C811B81AA81B981CE0FD11D0FB68A
:101BC000F894DEBF0FBECDBFED010895FB019F016C
:101BD00042306CF045325CF4642F772799DF805DEA
:101BE0008A330CF0895D8193CB010097A9F71082AD
:101BF000C90115C0E199FECF9FBB8EBBE09A992722
:101C00008DB30895262FE199FECF9FBB8EBB2DBBD0
:101C10000FB6F894E29AE19A0FBE01960895DC019E
:101C2000FC01672F71917723E1F7329704C07C9113
:101C30006D9370836291AE17BF07C8F30895F8944F
:021C4000FFCFD4
:101C4200370401000000000000000000010202034E
:101C52000303030404040404040404050505050540
:101C6200050505050505050505050506060606061D
:101C72000606060606060606060606060606060602
:101C820006060606060606060606060707070707ED
:101C920007070707070707070707070707070707D2
:101CA20007070707070707070707070707070707C2
:101CB20007070707070707070707070707070707B2
:101CC200070707070707070707070708080808089D
:101CD2000808080808080808080808080808080882
:101CE2000808080808080808080808080808080872
:101CF2000808080808080808080808080808080862
:101D02000808080808080808080808080808080851
:101D12000808080808080808080808080808080841
:101D22000808080808080808080808080808080831
:101D32000808080808080808080808080808080821
:0C1D42000808080808080808080808003D
:00000001FF
